:100000003928A000A00DA00D200D3839C1389F005F
:100010000030A100323020201F151F190D28A1012A
:100020001E083428A301A200FF30A207031CA30767
:10003000031C34280330A100DF3020201428A10144
:10004000E83EA000A109FC30031C2928A0070318E2
:100050002628A0076400A10F262820182F28A01CFE
:10006000332800003328080083130313831264002D
:100070000800FF2383168F00831283160F3085003C
:1000800002309F008312BB01BA010A3012200030F7
:100090000120BD000A30122001300120BC000A30CE
:1000A000122002300120BE0064003B08013C031D09
:1000B000622805303D07B200B301B30D0D303202A6
:1000C000C00064283D08C00064003A08013C031DDC
:1000D0006D280D303C07BF006F283C08BF0064004E
:1000E0003E084002031C842885168316851283125D
:1000F000BB0164003F083E02031C8F2805168316CF
:1001000005128312BA0145288512831685128312BF
:1001100005168316051283120130BB00452805120F
:100120008316051283120130BA0045286300962811
:02400E006C3F05
:00000001FF
